:10800000FEDF07EA000000000000000000000000A2
:108010000000000000000000000000000000000060
:108020000000000000000000000000000000000050
:108030000000000000000000000000000000000040
:108040000000000000000000000000000000000030
:02000004001FDB
:020000040020DA
:1000000002D3A0E3B40000EBFEFFFFEA001080E59E
:100010001EFF2FE1B010C0E11EFF2FE10010C0E570
:100020001EFF2FE1000090E51EFF2FE10E00A0E172
:100030001EFF2FE100C0A0E33ACF07EE4FF07FF59F
:1000400000C0A0E315CF07EE00C0A0E3D5CF07EEB8
:100050004FF07FF56FF07FF510FF2FE11EFF2FE1CE
:1000600000000FE11EFF2FE1100F11EE1EFF2FE128
:1000700010402DE908009FE5E9FFFFEB1040BDE8C7
:100080001EFF2FE15450213F10402DE91C009FE539
:10009000E3FFFFEB010010E3FBFFFF0A10009FE509
:1000A000DFFFFFEB1040BDE8FF0000E21EFF2FE185
:1000B0005450213F4050213F10402DE90C009FE556
:1000C000D7FFFFEB1040BDE8010000E21EFF2FE16B
:1000D0005450213F10402DE90040A0E11C009FE555
:1000E000CFFFFFEB200010E3FBFFFF0A0410A0E1AD
:1000F0000C009FE5C4FFFFEB1040BDE81EFF2FE1A1
:100100005450213F4050213F10402DE910009FE501
:10011000C3FFFFEB010C10E3FBFFFF1A1040BDE82B
:100120001EFF2FE15450213F70402DE90050A0E107
:100130002040A0E3044044E23504A0E10F0000E2C7
:10014000090050E33700808230008092E0FFFFEB2F
:10015000000054E3F6FFFF1A2000A0E37040BDE862
:10016000DBFFFFEA10402DE9EEFFFFEB0D00A0E3FF
:10017000D7FFFFEB0A00A0E31040BDE8D4FFFFEA81
:1001800010402DE90110A0E3D4009FE59EFFFFEB96
:100190000010A0E3CC009FE59BFFFFEB0010A0E365
:1001A000C4009FE598FFFFEB0310A0E3BC009FE5B0
:1001B00095FFFFEB0010A0E3B4009FE592FFFFEB7B
:1001C0000010A0E39C009FE58FFFFFEBC610A0E3AB
:1001D000A0009FE58CFFFFEB9C109FE59C009FE536
:1001E00089FFFFEB98009FE58DFFFFEB3F1AC0E30F
:1001F000121A81E388009FE583FFFFEB0010A0E364
:1002000080009FE580FFFFEB0040A0E30400A0E139
:10021000014084E290FFFFEB960054E3FAFFFF1ADF
:100220000319A0E360009FE577FFFFEB0040A0E328
:100230000400A0E1014084E287FFFFEB960054E355
:10024000FAFFFF1A0010A0E33C009FE56EFFFFEBF2
:100250000310A0E310009FE56BFFFFEB1040BDE82B
:100260001EFF2FE10450213F4450213F6050213FA9
:100270004C50213F5050213F4850213F0E0100007B
:100280006850213F0400203F9400203F9800203F09
:1002900010402DE91C409FE5F918A0E30400A0E1FF
:1002A00059FFFFEB0400A0E10C109FE556FFFFEBA8
:1002B0001040BDE81EFF2FE108B4003F0002F90026
:1002C00010402DE908009FE555FFFFEB1040BDE809
:1002D0001EFF2FE120B4003F1EFF2FE1F0472DE964
:1002E0000070A0E3FBFFFFEBA4FFFFEB6C029FE5B8
:1002F0009BFFFFEB4CFFFFEB99FFFFEB57FFFFEB83
:1003000097FFFFEB57FFFFEB95FFFFEB4900A0E3E3
:100310006FFFFFEB4800A0E36DFFFFEB4500A0E39C
:100320006BFFFFEB5800A0E369FFFFEB0D00A0E3BC
:1003300067FFFFEB0A00A0E30790A0E10760A0E1E0
:100340000750A0E10780A0E10740A0E160FFFFEBBC
:100350004CFFFFEB3A0050E32B00000A0A0050E389
:100360000D00501301A0A00300A0A0132900000A53
:100370002030C0E3470053E35000000A013044E25C
:10038000140053E303F19F97F0FFFFEAFC03200002
:10039000FC0320009C0420009C0420009C042000FE
:1003A0009C0420007C042000440420002004200041
:1003B0002004200020042000200420001404200039
:1003C000E0032000E0032000E0032000E003200021
:1003D000E0032000E0032000E0032000E003200011
:1003E000390050E3070040820992A0E10F0000E2CB
:1003F000150054E3099080E14C00000A21FFFFEB57
:100400003A0050E3014084E2D3FFFF1A0140A0E329
:10041000CEFFFFEA0662A0E10040A0E3CBFFFFEAC7
:10042000390050E3070040820662A0E10F0000E2BD
:10043000066080E10668A0E12668A0E1014084E250
:10044000C2FFFFEA390050E3070040820552A0E1F5
:100450000F0000E2055080E1FF5005E2010055E386
:100460002700000A0E40A033B8FFFF3A020055E310
:100470000940A0030040A013B4FFFFEA390050E395
:10048000070040820552A0E10F0000E2055080E124
:10049000FF5005E20840A0E3ACFFFFEA390050E35B
:1004A000070040820882A0E10F0000E2088080E19E
:1004B0000888A0E1288886E1014084E2A3FFFFEAE2
:1004C0000D00A0E302FFFFEB2D00A0E300FFFFEB18
:1004D0002D00A0E3FEFEFFEB0D00A0E3FCFEFFEB12
:1004E0000A00A0E3FAFEFFEB0A00A0E3F8FEFFEB30
:1004F0000209A0E3CEFEFFEB0A00A0E1F047BDE851
:100500001EFF2FE11440A0E30700A0E114FFFFEB62
:10051000014054E2FBFFFF1A0470A0E10490A0E147
:100520000460A0E10450A0E10480A0E187FFFFEA9D
:10053000693829E02334A0E1FF3CC3E3699423E058
:100540000800A0E1077088E00910A0E1AEFEFFEB13
:10055000077089E0048088E20E40A0E37BFFFFEA99
:040560007856341283
:040000030000800079
:00000001FF
